S024000062696E2F6F70656E626C745F6F6C696D65785F73746D3332683130332E73726563A3
S315080000005409002035260008192600081926000874
S3150800001019260008192600081926000819260008B6
S3150800002019260008192600081926000819260008A6
S315080000301926000819260008192600081926000896
S315080000401926000819260008192600081926000886
S315080000501926000819260008192600081926000876
S315080000601926000819260008192600081926000866
S315080000701926000819260008192600081926000856
S315080000801926000819260008192600081926000846
S315080000901926000819260008192600081926000836
S315080000A01926000819260008192600081926000826
S315080000B01926000819260008192600081926000816
S315080000C01926000819260008192600081926000806
S315080000D019260008192600081926000819260008F6
S315080000E019260008192600081926000819260008E6
S315080000F019260008192600081926000819260008D6
S3150800010019260008192600081926000819260008C5
S3150800011019260008192600081926000819260008B5
S3150800012019260008192600081926000819260008A5
S315080001301926000819260008192600081926000895
S315080001401926000819260008192600081926000885
S3150800015040F2F003C2F200031B78CBB94FF4805388
S31508000160C4F202039A6942F010029A614FF480536E
S31508000170C4F201035A6822F470425A605A6842F47B
S31508000180E0425A6040F2F003C2F2000301221A70FC
S3150800019001284FF48053C4F201034FF400620CBFE8
S315080001A05A611A61704700BF4FF48053C4F20203C4
S315080001B09A6942F004029A614FF40063C4F201039B
S315080001C01A6822F00F021A601A6842F004021A60CE
S315080001D0704700BF4FF40063C4F20103986880F0CB
S315080001E0010000F00100704700B583B000230093BA
S315080001F001934FF48053C4F202031A6842F00102D5
S315080002001A6059680022CFF6FF020A405A601A6837
S3150800021022F0847222F480321A601A6822F480224C
S315080002201A605A6822F4FE025A604FF41F029A6056
S315080002301A6842F480321A604FF48053C4F20203FB
S3150800024040F2DC52196801F400310191009901313C
S315080002500091019911B900999142F3D14FF4805355
S31508000260C4F202031B6813F4003F06D142F2906001
S31508000270C0F60000672101F08FFC4FF40053C4F26A
S3150800028002031A6842F010021A601A6822F0030282
S315080002901A601A6842F002021A604FF48053C4F2D8
S315080002A002035A685A605A6842F400525A605A68F9
S315080002B042F480625A605A6822F47C125A605A687C
S315080002C042F4E8125A601A6842F080721A604FF4D3
S315080002D08053C4F202031A6812F0007FFBD04FF471
S315080002E08053C4F202035A6822F003025A605A681D
S315080002F042F002025A604FF48053C4F202035A686D
S3150800030002F00C02082AFAD14FF48053C4F2020311
S315080003105A6822F480025A60DA6942F40002DA6105
S3150800032001F0E4F901F0F0F9FCE700BF08B501F0C7
S31508000330F1FD08BD08B501F049FE08BD08B540F253
S31508000340F403C2F200031B68052B01D101F0E2FD9C
S3150800035008BD00BF40F22873C2F200039B7A2BB196
S3150800036040F2F403C2F2000305221A60704700BF88
S3150800037040F2F403C2F2000304221A60704700BF79
S31508000380704700BF704700BF10B5062810D140F26D
S315080003904873C2F200031B681A7802F07F02012A2A
S315080003A008D15A7942B99A78212A07D0022010BD75
S315080003B0022010BD022010BD022010BD40F20D52D1
S315080003C0C0F600029A6100245C82204600F09EF87E
S315080003D0204610BD0220704721B9002814BF02200C
S315080003E0002070470220704710B501F01FFE40F24A
S315080003F04873C2F200031B6800249C7200F0E4F8FC
S3150800040001F04EF940F2F403C2F200031C6010BD7D
S3150800041010B540F24873C2F200031B6800249C72B0
S3150800042042F2D862C0F60002D2795A72DC722046CD
S3150800043000F0F8FF20464FF4007100F0FDFF20465B
S31508000440102101F005F82046402101F0A7F82046C2
S31508000450802101F091F8204601F056F840F2080391
S31508000460C2F20003204693F82C1001F0DBF8204670
S3150800047001F038F80120214600F0DEFF01204FF494
S31508000480807101F079F80120C02101F087F8012078
S31508000490402101F0B7F80120402101F0C3F80120FE
S315080004A04FF4405100F0F0FF0120202100F0D0FF6A
S315080004B0204600F09BFD40F2F403C2F2000301223D
S315080004C01A6010BD08B540F26401C2F2000100F0DE
S315080004D0DFFA08BD08B540F20001C2F2000100F0DB
S315080004E0D7FA08BD08B540F24873C2F200031B6884
S315080004F0D978052908D840F26C03C2F2000303EB49
S31508000500C10100F0C5FA08BD002008BD08B540F2D3
S315080005105C01C2F2000100F0BBFA08BD08B545F659
S315080005204443C4F200031A6892B240F21473C2F24A
S3150800053000031A801A8840F24C73C2F200031B8823
S31508000540134003F400739BB283B145F64443C4F2E7
S3150800055000034FF6FF521A6040F2F103C2F200039D
S315080005601A780132D2B21A70FFF7E8FE40F2147315
S31508000570C2F200031A8840F24C73C2F200031B88C9
S31508000580134003F400439BB20BB100F0B3FD40F2F5
S315080005901473C2F200031A8840F24C73C2F20003C5
S315080005A01B88134003F480639BB263B145F644434A
S315080005B0C4F200034FF6FF321A6040F20803C2F293
S315080005C000035B68984708BD08B50120FFF7C0FD22
S315080005D045F64043C4F2000301221A6040F24C7209
S315080005E0C2F200020020186045F64441C4F2000138
S315080005F008604FF4E0511180196008BD08B538B994
S3150800060040F24873C2F200031B6801221A8208BD31
S3150800061040F24473C2F200031B681B68984740F215
S315080006204873C2F2000318680A3008BD08B538B91D
S3150800063040F24873C2F200031B6801221A8208BD01
S3150800064040F24473C2F200031B689B68984740F265
S315080006504873C2F2000318680C3008BD08B538B9EB
S3150800066040F24873C2F200031B6802221A8208BDD0
S3150800067040F21873C2F2000300221A8040F248734F
S31508000680C2F200031A68137813F07F0317D1537A5E
S3150800069013F0200F1FBF40F21872C2F200020221A7
S315080006A0117013F0400F40F21873C2F200031A7863
S315080006B014BF42F0010222F001021A702BE0012B4E
S315080006C035D0022B38D1537903F00F0213F0800F7F
S315080006D010D0920002F1804202F5B842136803F086
S315080006E03003102B17D140F21873C2F2000301220F
S315080006F01A7010E0920002F1804202F5B8421368BF
S3150800070003F44053B3F5805F01BF40F21873C2F299
S31508000710000301221A7040F24473C2F200031B68F8
S315080007201B69984740F21870C2F2000008BD40F2F3
S315080007301870C2F2000008BD002008BDF8B540F2E6
S315080007404873C2F200031C68238A227A002B08BF6A
S31508000750042A29D140F2F803C2F200031B78012BC0
S315080007601AD145F65043C4F200031A6892B243F20E
S315080007700203C2F2000313445B0000221A6040F22F
S315080007805073C2F200033021198040F2F803C2F216
S3150800079000031A70042632E040F25073C2F20003D6
S315080007A010221A8007262AE0A58AAB428CBF0226A9
S315080007B004269D4228BF1D46A36928469847074632
S315080007C0002000F0FFFE014638462A4600F000FEEB
S315080007D00020294600F016FF238A5B1B2382638AC2
S315080007E01D44658240F25073C2F2000330221A801B
S315080007F040F24E73C2F200034FF440521A8040F2A0
S315080008004873C2F200031B681E72F8BD08B540F2B1
S315080008104873C2F200031A68D17840F29403C2F210
S3150800082000035B788B420DD393786BB993886BB9C9
S31508000830917240F24473C2F200031B685B689847E2
S31508000840002008BD022008BD022008BD022008BD00
S3150800085010B540F24874C2F20004226840F22073D0
S31508000860C2F200031B689B695079D17898472368C0
S315080008709A7A92B198B91A799AB99B789BB940F243
S315080008804473C2F200031B68DB68984723685A79E9
S31508000890DA72DA781A73002010BD022010BD022021
S315080008A010BD022010BD022010BD00BF10B540F2D9
S315080008B04873C2F200031A68137813F07F0305D150
S315080008C0537A23F020035372002010BD022B6FD1F8
S315080008D05388002B6ED11379002B6DD1517921F0F5
S315080008E0800011F0800F4FEA800303F1804303F57F
S315080008F0B84319BF1C6804F030041B6803F440545D
S3150800090040F29403C2F200031B78984256D2002C98
S3150800091056D0937A002B55D011F0800F12D0830051
S3150800092003F1804303F5B8431B6803F03003102B2B
S3150800093035D1C4B2204600F00BFE2046302100F027
S3150800094087FD2CE0840004F1804404F5B84423684C
S3150800095003F44053B3F5805F21D198B940F20803F8
S31508000960C2F2000393F82C1000F05CFE22684BF6E6
S315080009708F73134083F4405343F4004343F08003DA
S3150800098023600CE000F0D0FD22684BF68F7313400D
S3150800099083F4405343F4004343F08003236040F25A
S315080009A04473C2F200031B685B699847002010BDB8
S315080009B0022010BD022010BD022010BD022010BD6D
S315080009C0022010BD022010BD10B540F24873C2F2D5
S315080009D000031868427922F0800112F0800F4FEA6E
S315080009E0810303F1804303F5B84319BF1C6804F07B
S315080009F030041B6803F4405440F29403C2F2000327
S31508000A001B78994227D243883BBB44B3837A43B3C6
S31508000A1012F0800F4FEA810202F1804202F5B842D5
S31508000A2011681DBF48F6BF730B4083F010034BF6E1
S31508000A308F7304BF0B4083F4805343F4004343F0A1
S31508000A408003136040F24473C2F200031B689B697B
S31508000A509847002010BD022010BD022010BD0220BC
S31508000A6010BD022010BD00BF08B540F24873C2F29F
S31508000A7000031B685A7A42F020025A7240F2447305
S31508000A80C2F200031B68DB699847002008BD00BF57
S31508000A9040F24873C2F200031B685A8A18B989885B
S31508000AA08A1A1A82704708681044704708B540F2D7
S31508000AB00803C2F20003002093F82C1000F0B2FDE0
S31508000AC040F24873C2F200031B68187A08280CD152
S31508000AD040F24E73C2F200034FF480521A8040F27D
S31508000AE05073C2F2000310221A80092814BF00208E
S31508000AF0012008BD70B582B045F65043C4F2000324
S31508000B001A6892B243F20403C2F2000313445B006C
S31508000B101D6840F24873C2F200031B681A7A092A54
S31508000B201BD0ADB26D0005F1804505F5C0452A78A4
S31508000B301A7040F24874C2F2000423686A785A7040
S31508000B402668A88800F0A6FD70802668288900F027
S31508000B50A1FDB080AA892368DA8040F24873C2F200
S31508000B6000031B6801221A72DA88002A77D15C789A
S31508000B701A7812F07F022ED1092C02D1FFF746FE11
S31508000B803BE0052C0FD193F90320002AB8BF0822B1
S31508000B905EDB9A78002A55D19A88002A54D19B7A26
S31508000BA0002B39D052E0032C07D1DA78012A25D157
S31508000BB09B881BBBFFF758FF1FE0012C1ED1DA7874
S31508000BC0012A1BD19A88CAB95B7A13F0200F15D06F
S31508000BD0FFF76CFE11E0012A04D10B2C0ED1FFF7AA
S31508000BE037FE0AE0022A09D1012C02D1FFF75EFE80
S31508000BF003E0032C02D1FFF7E7FE68B140F2207349
S31508000C00C2F200031B685B6920469847032808BFA1
S31508000C1009221DD00822D8B945F65043C4F200036C
S31508000C201A6892B243F20203C2F2000313445B004D
S31508000C3000221A6040F25073C2F2000330221A8072
S31508000C40062205E0082203E0082201E00822FFE761
S31508000C5040F24873C2F200031B681A7217E15A7809
S31508000C60062A21D11A7812F07F0F40F0A9809B78C6
S31508000C70012B06D140F22073C2F200031B68DA6921
S31508000C808DE0022B06D140F22073C2F200031B68E6
S31508000C901A6A84E0032B40F0938040F22073C2F274
S31508000CA000031B685A6A7AE0002A52D15A88002A39
S31508000CB040F086805A6822F47F42B2F5003F7FD121
S31508000CC01A7812F07F0204D19B88002B00F0E2808C
S31508000CD076E0012A14D140F22072C2F200021268AC
S31508000CE09269587900219047002869D140F24873E3
S31508000CF0C2F200031B689B7A002B40F0D0805FE0AD
S31508000D00022A5DD15A7902F00F0112F0800F4FEADC
S31508000D10810303F1804303F5B84319BF186800F04F
S31508000D2030001B6803F4405040F29403C2F20003FB
S31508000D301B78994244D212F0700F14BF0023012386
S31508000D4000280CBF002003F00100002840F0AC800A
S31508000D5036E0082A05D11B7813F07F0F00F0A9802A
S31508000D602EE00A2A2CD11A7802F07F02012A27D10E
S31508000D709A7A2AB35A881ABB5A6822F47F42B2F57D
S31508000D80803F1DD140F22072C2F2000212689269B9
S31508000D90587900219047002800F0908010E07AB139
S31508000DA040F24874C2F200042368002058829A610F
S31508000DB0904723681A8A4FF6FF718A4226D120E0A7
S31508000DC040F22073C2F20003196840F24873C2F277
S31508000DD000031A680B6950789847032807D140F230
S31508000DE04873C2F200031B6809221A724FE040F2E8
S31508000DF04873C2F200031B681A8A4FF6FF718A42CB
S31508000E0002D109221A7242E0022800D012B9082239
S31508000E101A723CE093F9001000292FDAD98801915B
S31508000E200198824202D9019A1A821CE091421AD983
S31508000E3040F22071C2F20001096891F82C10914223
S31508000E4006D940F2F802C2F20002002111700AE047
S31508000E5092FBF1F001FB10222AB940F2F802C2F225
S31508000E6000020121117040F22072C2F200021268DB
S31508000E7092F82C209A82FFF761FC08E003221A7286
S31508000E8040F24E73C2F200034FF440521A80FFF745
S31508000E900DFE18E040F25D62C0F6000280E740F2FF
S31508000EA05D62C0F600027BE740F25D62C0F60002B2
S31508000EB076E740F2FD52C0F6000271E740F22D6275
S31508000EC0C0F600026CE702B070BD00BF70B540F214
S31508000ED04873C2F200031C68237A022B18BF042B3E
S31508000EE008BF082274D0032B18BF052B63D1228AAA
S31508000EF0A369ABB1A2B1A58A954228BF1546284673
S31508000F0098470646238A5B1B2382638A2B4463829F
S31508000F10002000F067FB014630462A4600F072FAC8
S31508000F20238A002B5DD040F24E73C2F200034FF4C1
S31508000F3040521A800020014600F064FB40F25073CC
S31508000F40C2F2000330221A80238AA28A9A4207D85C
S31508000F5040F24873C2F200031B6803221A7223E0A8
S31508000F603BB140F24873C2F200031B6805221A72AD
S31508000F701AE040F24873C2F200031B6806221A728E
S31508000F8045F65043C4F200031A6892B243F20203CC
S31508000F90C2F2000313445B0000221A6040F2507349
S31508000FA0C2F2000330221A8040F24873C2F20003EC
S31508000FB01B681A7A0CE0072B18BF082208D140F2E2
S31508000FC02073C2F200031B68DB6898470822FFE714
S31508000FD040F24873C2F200031B681A72FFF766FDF7
S31508000FE070BDA38A002BC4D1B2E700BF70B440F22B
S31508000FF09403C2F200031D789DB1002340F60F76D4
S31508001000DAB2910001F1804101F5B8410C6842F469
S31508001010004242F08002344022430A6001339D4276
S31508001020EED840F0800045F64C43C4F20003186041
S3150800103070BC704708B540F24873C2F200031A68DC
S31508001040137A022B18BF042B08D1FFF777FB40F25F
S315080010504873C2F200031B681A7A1DE0062B18BFF4
S31508001060082219D15378052B0DD1137813F07F0F69
S3150800107009D1D078FFF7BAFF40F24473C2F20003F1
S315080010801B681B6A984740F22073C2F200031B686C
S315080010909B6898470822FFE740F24873C2F20003AC
S315080010A01B681A72FFF702FD08BD00BF704700BF34
S315080010B008B540F24872C2F2000240F22873C2F242
S315080010C00003136002221A7240F22072C2F2000272
S315080010D040F20803C2F20003136040F24472C2F2FF
S315080010E0000240F23801C2F2000111601B689847FD
S315080010F008BD00BF2DE9F04383B00023ADF80630E4
S3150800110045F64447C4F2000740F21474C2F20004DC
S3150800111040F22476C2F2000640F2B408C2F2000891
S3150800112040F2D009C2F2000940F24E75C2F200053B
S3150800113043E1238803F00F033370002B40F00F813F
S315080011404FF4B843C4F200031A6892B22A80298879
S3150800115001F0300140F25072C2F2000211802A8872
S3150800116002F440522A8019684BF6BF720A4082F48C
S31508001170005282F0200242F4004242F080021A60D5
S31508001180238803F010039BB2002B46D14FF4B844D2
S31508001190C4F20004226848F60F7313402360FFF771
S315080011A049FF22684BF6BF73134040F24E72C2F2F3
S315080011B00002128802F4805292B20AB183F4805374
S315080011C040F24E72C2F20002128802F4005292B243
S315080011D00AB183F4005340F25072C2F20002128838
S315080011E002F0100292B20AB183F0100340F2507274
S315080011F0C2F20002128802F0200292B20AB183F00B
S31508001200200348F28002CFF6FF721A4392B24FF4D7
S31508001210B843C4F200031A60D6E04FF4B843C4F2E8
S3150800122000031B689BB2ADF80630BDF8063003F420
S3150800123000639BB2002B46D04FF4B844C4F20004B6
S31508001240226840F68F7313402360FFF753FC226829
S315080012504BF6BF73134040F24E72C2F20002128878
S3150800126002F4805292B20AB183F4805340F24E726D
S31508001270C2F20002128802F4005292B20AB183F452
S31508001280005340F25072C2F20002128802F01002B5
S3150800129092B20AB183F0100340F25072C2F2000211
S315080012A0128802F0200292B20AB183F0200348F2B3
S315080012B08002CFF6FF721A4392B24FF4B843C4F2D3
S315080012C000031A6080E0BDF806301BB2002B74DA02
S315080012D04FF4B844C4F20004226840F68F731340F2
S315080012E02360FFF7F3FD22684BF6BF73134040F205
S315080012F04E72C2F20002128802F4805292B20AB109
S3150800130083F4805340F24E72C2F20002128802F44D
S31508001310005292B20AB183F4005340F25072C2F2FC
S315080013200002128802F0100292B20AB183F010038A
S3150800133040F25072C2F20002128802F0200292B203
S315080013400AB183F0200348F28002CFF6FF721A43EF
S3150800135092B24FF4B843C4F200031A6034E09B001B
S3150800136003F1804303F5B8431A6892B2ADF8062034
S31508001370BDF8062012B2002A09DA196840F68F72FB
S315080013800A401A603378013B59F823309847BDF86C
S31508001390063003F080039BB27BB13278920002F1EB
S315080013A0804202F5B842116848F60F730B40136085
S315080013B03378013B58F8233098473B689AB2228025
S315080013C013F4004F7FF4B5AE03B0BDE8F08300BF59
S315080013D010B4531C01F1005101F5405252005B1044
S315080013E00DD00432023010F8014C10F8021C41EA04
S315080013F0042122F8041C04320230013BF3D15DF8C3
S31508001400044B7047013201F1005101F54051490082
S31508001410531005D051F8042B20F8022B013BF9D1C3
S31508001420704700BF4FF6F873034045F65042C4F2C2
S3150800143000021360704700BF800000F1804202F589
S31508001440B842106848F68F13034019431160704775
S31508001450800000F1804202F5B842106848F6BF7372
S31508001460034001F0100080B208B183F0100301F0C8
S31508001470200189B209B183F0200343F4004343F005
S3150800148080031360704700BF800000F1804202F5B8
S31508001490B84210684BF68F73034001F4805080B24F
S315080014A008B183F4805301F4005189B209B183F479
S315080014B0005343F4004343F080031360704700BFB2
S315080014C0800000F1804202F5B842116848F6BF7301
S315080014D00B4083F0300343F4004343F0800313606A
S315080014E0704700BF800000F1804202F5B8421168DB
S315080014F04BF68F730B4083F4405343F4004343F099
S3150800150080031360704700BF800000F1804202F537
S31508001510B842116840F60F630B4043F4004343F0AA
S3150800152080031360704700BF800000F1804303F515
S31508001530B8431A6812F4804F08D0196840F60F723B
S315080015400A4042F4404242F080021A60704700BFE7
S31508001550800000F1804303F5B8431A6812F0400F83
S3150800156008D0196840F60F720A4042F4004242F069
S31508001570C0021A60704700BF45F65043C4F2000324
S315080015801A684FF6FE730B4092B202EBC00000F1E8
S31508001590005202F5405252001360704745F6504318
S315080015A0C4F200031B684FF6FE720A409BB203EBB7
S315080015B0C00043F20403C2F2000303445B001A604E
S315080015C0704700BF45F65043C4F200031B689BB240
S315080015D003EBC00000F1005303F540535B00188885
S315080015E0704700BF45F65043C4F200031B689BB220
S315080015F003EBC00043F20403C2F2000303445B009A
S315080016001888704745F65043C4F200031B689BB21E
S3150800161003EBC00043F20203C2F2000303445B007B
S315080016201960704745F65043C4F200031B689BB225
S3150800163003EBC00043F20603C2F2000303445B0057
S315080016403E290BD94A0911F01F0F04BF02F1FF32D8
S3150800165092B2920242F400421A6070474A0811F0A8
S31508001660010F1CBF013292B292021A60704700BF86
S3150800167045F65043C4F200031B689BB203EBC00057
S3150800168043F20603C2F2000303445B001868C0F382
S3150800169009007047C3B2000A40EA0320704700BF3A
S315080016A045F64443C4F200030020186040F24C7328
S315080016B0C2F200034FF406421A8045F64043C4F2CC
S315080016C000031A60704700BF70B50E4600F07F052C
S315080016D02846FFF7CDFF04462846FFF783FF014655
S315080016E030462246FFF78EFE204670BD08B500F04C
S315080016F057FA00F04DFA00F0D7FC00F0B7FC00F0FE
S315080017000DF800F039FA08BD08B500F043FA00F004
S31508001710E7FC00F00FF800F039FA08BD08B500F04C
S3150800172059F800F0FDFA40F2EC03C2F20003022277
S315080017301A7008BD08B540F2FC00C2F2000000F0BD
S3150800174089FB01280BD140F2EC03C2F20003022206
S315080017501A7040F2FC00C2F2000000F051F808BD11
S3150800176008B500F033FB08BD08B540F2EC03C2F239
S3150800177000031B78022B02D1C9B200F02DFB00F042
S3150800178037F808BD40F2EC03C2F200031B78012BC0
S3150800179001D9032B01D1002070473F20704700BFB5
S315080017A040F2EC03C2F200031B78012B01D9032B8C
S315080017B001D1002070473F20704700BF40F23C131C
S315080017C0C2F20003FE22DA7018710222A3F844203E
S315080017D0704700BF40F23C13C2F2000300221A70A1
S315080017E09A6483F84220A3F844209A705A70704786
S315080017F040F23C13C2F20003002283F842207047ED
S3150800180038B504460178FF291CD140F23C14C2F2CF
S3150800181000040023637001252570FF22E270102260
S3150800182022716371FFF7AEFFA071FFF7B9FFE07190
S31508001830FFF7B6FF000A20726572A5720823A4F89E
S31508001840443079E140F23C13C2F200031B78012BC5
S3150800185040F09081C939352900F26B81DFE811F033
S31508001860DB00690169016501690169015901FC002B
S3150800187042012F016901690169016901690169016B
S3150800188069016901690169016901690169016901FA
S3150800189069016901690169016901690169016901EA
S315080018A069016901690169016901690169016901DA
S315080018B0690169017F0054003600730069016901F6
S315080018C06901A1006901B900BD00CE004578FFF79E
S315080018D059FF0138854203DD2220FFF76FFF2BE110
S315080018E040F23C15C2F20005281DA96C627800F08A
S315080018F075F9FF23EB706278AB6C1344AB646378BD
S315080019000133A5F8443017E14578FFF73BFF013866
S31508001910854203DD2220FFF751FF0DE1616840F2A1
S315080019203C15C2F20005A964281D627800F056F934
S31508001930FF23EB706278AB6C1344AB6463780133B6
S31508001940A5F84430F8E040F23C13C2F20003FF2247
S31508001950DA7042689A640122A3F84420ECE040F267
S315080019603C13C2F20003FF22DA709B6C406840B158
S315080019701844002213F8011B0A44D2B28342F9D153
S3150800198000E0002240F23C13C2F20003C3F807202D
S3150800199001221A7100225A719A710822A3F844206A
S315080019A0CAE040F23C13C2F20003FF22DA7042F2A8
S315080019B04072C0F600029A6400221A715A719A712E
S315080019C00721D9711A725A729A720822A3F844200A
S315080019D0B2E00020FFF7F2FEAEE040F23C13C2F29E
S315080019E00003FF22DA7000221A71597859719A7128
S315080019F0DA711A720622A3F844209DE040F23C13DD
S31508001A00C2F2000300221A705A70FF22DA7001220D
S31508001A10A3F8442090E040F23C13C2F200039D6C08
S31508001A20FFF7B0FE411E2846621C00F023FB18B9DA
S31508001A303120FFF7C3FE7FE040F23C14C2F20004F7
S31508001A40FF23E370A56CFFF79DFE013D2844A064C3
S31508001A500123A4F844306FE04578FFF793FE023877
S31508001A60854203DD2220FFF7A9FE65E040F23C131C
S31508001A70C2F20003FF22DA700122A3F8442061783B
S31508001A8039B900F007FB002856D13120FFF796FE3A
S31508001A9052E040F23C13C2F20003986CA21C00F01C
S31508001AA0E9FA18B93120FFF789FE45E040F23C1300
S31508001AB0C2F2000361789A6C0A449A643CE040F2E8
S31508001AC03C14C2F20004FF23E370002525716571FA
S31508001AD0FFF758FEA071E571257265720723A4F811
S31508001AE0443029E040F23C13C2F20003986C616866
S31508001AF000F0C4FA18B93120FFF760FE1CE040F286
S31508001B003C13C2F20003FF22DA700122A3F8442034
S31508001B1012E000F049F840F23C13C2F20003FF223B
S31508001B20DA700122A3F8442006E03120FFF746FECA
S31508001B3002E02020FFF742FE40F23C13C2F2000307
S31508001B4093F84230012B02D11020FFF737FE40F2FE
S31508001B503C13C2F20003B3F844100BB2002B09DDA4
S31508001B6040F23C10C2F20000012380F842300330F4
S31508001B70FFF7FAFD38BD00BF08B5FEF715FBFEF7FF
S31508001B8029FB08B900F010F808BD00BF704700BF70
S31508001B90704700BF704700BF08B5FFF7FBFFFCE7BB
S31508001BA008B500F043FD08BD10B500F06BFAA0B10A
S31508001BB0FFF7D6FD00F08CFA00F068FA20F06040D6
S31508001BC020F07F004EF60853CEF20003186000F0AE
S31508001BD05DFA446800F02CFDA04710BD70B5561E8E
S31508001BE0B6B24AB14C1E0E44451A14F8013F2B559D
S31508001BF0FFF7D0FFB442F8D170BD00BF30B492B140
S31508001C004B1C0331541EE4B201EB44040021020FBD
S31508001C10092A94BF3032373203F8012C000103F841
S31508001C20021BA342F3D130BC704700BF38B5044647
S31508001C300D46012807D942F24870C0F600004FF455
S31508001C40FC71FFF7A9FF40F2D013C2F2000304EBC0
S31508001C50440203EBC2035A7C1B7C9A4220D040F212
S31508001C60D013C2F2000304EB440203EBC203DA68A2
S31508001C701570597C01315974DA680132DA605B688B
S31508001C809A420FD940F2D013C2F20003620011192A
S31508001C9053F83110144403EBC403D960012038BD4E
S31508001CA0002038BD012038BD38B504460D46012848
S31508001CB007D942F24870C0F6000040F21A21FFF731
S31508001CC06BFF40F2D013C2F2000304EB440203EBAD
S31508001CD0C2035B7CFBB140F2D013C2F2000303EBF4
S31508001CE0C2039A6812782A70597C013959749A681D
S31508001CF001329A605B689A420FD940F2D013C2F259
S31508001D0000036200111953F83110144403EBC4039D
S31508001D109960012038BD002038BD012038BD00BFBC
S31508001D2010B540F2D013C2F200030020987403F1F4
S31508001D3018025A61012183F82A10D86240F2CC11A0
S31508001D40C2F200010A604021197440F2C421C2F2AD
S31508001D5000014C1C9C60DC6058741C6001F1400456
S31508001D605C6008705AB340F2CC11C2F20001D86A1E
S31508001D700860402183F8281040F20021C2F20001D1
S31508001D80481C18625862002483F82940986101F1BA
S31508001D9040035360927C0A7040F2C423C2F20003E7
S31508001DA01B78FF2B01D0FF2A06D142F24870C0F6F5
S31508001DB000007A21FFF7F0FEFFF77AF910BD40F22E
S31508001DC00023C2F20003FF221A70EEE708B50020CE
S31508001DD0FEF7BEF908BD00BF2DE9F84307460C46D5
S31508001DE03F2906D942F24870C0F600009921FFF74C
S31508001DF0D3FE40F2C423C2F2000318782146FFF747
S31508001E0015FF012806D042F24870C0F600009D2151
S31508001E10FFF7C2FE2646D4B1002440F2C425C2F21A
S31508001E20000542F24878C0F600084FF0A609FFF709
S31508001E30B1FE2878395DFFF7F9FE012803D0404640
S31508001E404946FFF7A9FE0134A3B2B342EFD3BDE872
S31508001E50F88300BF10B50446FEF760FB40F2C813CE
S31508001E60C2F200031B7803BB40F20023C2F2000350
S31508001E70187840F28811C2F20001FFF715FF012811
S31508001E803ED140F28813C2F200031B78002B39D0EA
S31508001E9040F2C813C2F2000301221A7040F2C913B5
S31508001EA0C2F200030020187010BD40F20023C2F2EF
S31508001EB0000340F2C912C2F2000211781878144BD6
S31508001EC01944FFF7F1FE01281ED140F2C913C2F2E8
S31508001ED000031A780132D2B21A7040F28813C2F29D
S31508001EE000031B78934211D120460949FFF776FE75
S31508001EF040F2C813C2F2000300221A70012010BD76
S31508001F00002010BD002010BD002010BD002010BD0F
S31508001F10890100202DE9F04383B040F2C423C2F2C0
S31508001F2000031C78012C07D942F24870C0F600005D
S31508001F3040F23A21FFF730FE40F2D013C2F2000316
S31508001F4004EB440403EBC4035B7C002B3BD0402B1F
S31508001F5034BF99464FF04009B9F1000F23D040F23B
S31508001F608423C2F200035C1E09F1FF36F6B21E4452
S31508001F7040F2C425C2F2000542F24877C0F60007CF
S31508001F8040F2491828780DF10701FFF78DFE012860
S31508001F9003D038464146FFF7FFFD9DF8073004F8A1
S31508001FA0013FB442EED140F28420C2F200004FF461
S31508001FB080714A46FFF70CFA01204946FFF722FBD3
S31508001FC00120FFF77DFA03B0BDE8F0832DE9F04163
S31508001FD0012040F24421C2F20001FFF775FB80B2EE
S31508001FE0F0B140F24423C2F200035C1E013886B207
S31508001FF01E4440F20025C2F2000542F24877C0F6B8
S3150800200000074FF4B778287814F8011FFFF70EFE7B
S31508002010012803D038464146FFF7BEFDB442F2D147
S315080020200120FFF75FFABDE8F08100BF38B54FF22F
S31508002030E873C1F6FF731B684FF2EC72C1F6FF72C4
S3150800204014684FF2F072C1F6FF721268D0180AD0FF
S31508002050054D29460822FFF7D1FD204605F1100156
S315080020600422FFF7CBFD38BD9A00002008B500F022
S3150800207051F908BD08B500F05BF908BD08B500F0D0
S315080020807FF908BD08B500F067FA08BD08B500F085
S31508002090BDFA08BD08B500F033FA10B100F090FAA1
S315080020A008BD002008BD00BF4EF21003CEF20003A3
S315080020B000221A6041F63F11C0F2010159609A6088
S315080020C00521196040F20833C2F200031A6070470E
S315080020D04EF21003CEF2000300221A60704700BFCA
S315080020E04EF21003CEF200031B6813F4803F1FBFA5
S315080020F040F20833C2F200031A68013218BF1A60A8
S31508002100704700BF4FF40053C4F202031A6942F045
S3150800211080021A61704700BFF8B5074600242546B5
S3150800212042F27076C0F60006FFF734FDA359BB42AB
S315080021300ED8311949680B449F4209D242F270738E
S31508002140C0F6000305EB450203EB8203187AF8BDD7
S3150800215001350C349C2CE7D1FF20F8BD2DE9F84356
S3150800216080460068FFF7D8FFFF285CD04FF400537D
S31508002170C4F2020340F22312C4F267525A6048F6C8
S31508002180AB12CCF6EF525A603422DA60DB6813F0F1
S31508002190010F04D0FFF7B6FF0020BDE8F8834FF41F
S315080021A00053C4F202031A6942F001021A610025BB
S315080021B008F104094FF40054C4F20204D8F80030B8
S315080021C0EF1859F80560B2B2EA52E36813F0010F46
S315080021D005D0FFF7DFFCE36813F0010FF9D1330CE4
S315080021E07B80E36813F0010F05D0FFF7D3FCE368A3
S315080021F013F0010FF9D13B68B34204D10435B5F5A4
S31508002200007FDBD101E0002400E001244FF40053F5
S31508002210C4F202031A6922F001021A61FFF772FF7B
S315080022202046BDE8F8830020BDE8F88338B50446A3
S315080022300D4640F20C33C2F20003984209D04FF41F
S31508002240C043C0F6000399420BD0FFF787FF20B9B9
S3150800225017E040F21054C2F20004C5F3080393B91C
S3150800226003E040F20C34C2F2000423689D420CD00D
S31508002270204640F8045B29464FF40072FFF7AEFC8F
S3150800228003E0002038BD002038BD204638BD00BF19
S315080022902DE9F04106460C4617461D464FEA5128D9
S315080022A04FEA48280368B3F1FF3F06D140F8048B8C
S315080022B041464FF40072FFF791FC3368434505D059
S315080022C030464146FFF7B2FF0646D0B13368E41AF6
S315080022D03444043408F50078FFF75CFC331DE31A30
S315080022E0B3F5007F06D330464146FFF79FFF064603
S315080022F050B1041D17F8013B04F8013B013DEBD131
S3150800230005E00020BDE8F0810020BDE8F08101204D
S31508002310BDE8F08140F21053C2F200034FF0FF32DD
S315080023201A6040F20C33C2F200031A60704700BF0D
S3150800233070B504460D461646FFF7EEFEFF281BD07D
S31508002340681E2044FFF7E8FEFF2817D0620A4FF4FC
S31508002350C043C0F60003B3EB422F07BF40F20C3070
S31508002360C2F2000040F21050C2F200002146324686
S315080023702B46FFF78DFF70BD002070BD002070BD95
S315080023802DE9F84304460E46FFF7C6FE0546701EBD
S315080023902044FFF7C1FE0446FF2D18BFFF2800F0B2
S315080023A0AB80854200F29F80022D40F29F800F2865
S315080023B000F29F804FF40053C4F2020340F2231246
S315080023C0C4F267525A6048F6AB12CCF6EF525A601E
S315080023D03422DA60DB6813F0010F04D0FFF792FEAF
S315080023E00020BDE8F8834FF40053C4F202031A69CB
S315080023F042F002021A6142F27079C0F600094F46AD
S315080024000026FFF7C7FB3B7AAB4208D142F270734E
S31508002410C0F6000306EB460253F8227005E00136C3
S315080024200C370D2EEDD14FF0FF37C8460025FFF7C4
S31508002430B1FB98F80830A34208D142F27073C0F68F
S31508002440000305EB450253F8228006E0013508F142
S315080024500C080D2DEBD14FF0FF384E460025FFF73F
S3150800246099FB337AA34209D142F27073C0F600038E
S3150800247005EB450203EB82035B6804E001350C3685
S315080024800D2DECD10023C7EB08084344C3F38F2373
S31508002490E3B1013B9EB20136B60200254FF4005463
S315080024A0C4F20204EB196361236943F04003236114
S315080024B0E36813F0010F05D0FFF76CFBE36813F030
S315080024C0010FF9D105F58065B542EBD14FF40053FC
S315080024D0C4F202031A6922F002021A61FFF712FE19
S315080024E00120BDE8F8830020BDE8F8830020BDE898
S315080024F0F8830020BDE8F8830020BDE8F88300BF14
S3150800250000B583B040F20C33C2F200031B68B3F186
S31508002510FF3F08BF01201CD040F20C33C2F2000373
S3150800252099685A681144DA6811441A6911445A6953
S3150800253011449A690A44D96953185B4202AA42F8B7
S31508002540043D46F25010C0F600000421FFF7F0FEE5
S31508002550FFE703B05DF804FB46F20402C0F600028A
S315080025604FF4C043C0F6000310681B68184446F2CF
S315080025700803C0F600031B68184446F20C03C0F6AD
S3150800258000031B68184446F21003C0F600031B68D4
S31508002590184446F21403C0F600031B68184446F2B2
S315080025A01803C0F600031B68184446F25013C0F619
S315080025B000031B681844D0F1010038BF002070479B
S315080025C008B540F20C33C2F200031B68B3F1FF3FB3
S315080025D006D040F20C30C2F20000FFF7BFFD88B10A
S315080025E040F21053C2F200031B68B3F1FF3F0BD051
S315080025F040F21050C2F20000FFF7B0FD003018BFDD
S31508002600012008BD002008BD012008BD4FF4C040C8
S31508002610C0F60000704700BF08B542F60C00C0F6C9
S3150800262000003121FFF7B8FA08BD00BF72B670473F
S3150800263062B6704710B540F20002C2F2000240F2DC
S31508002640ED03C2F200039A4210D2131D0D4CE41A90
S3150800265024F0030404340023104642F63C01C0F675
S3150800266000015A581A500433A342FAD106480749BA
S315080026704FF000028842B8BF40F8042BFADBFDF79A
S31508002680B3FD10BDF0000020F00000205207002026
S315080026906D61696E2E630000120110010000004092
S315080026A0501DAC6000010102030100000403090487
S315080026B02603570069006E005500530042002000AB
S315080026C0420075006C006B0020004400650076002F
S315080026D0690063006500000009022000010100C0CE
S315080026E0320904000002FF000004070581024000C9
S315080026F000070501024000001A034F00700065003C
S315080027006E0042004C00540020005500730065001E
S31508002710720000002C03570069006E005500530034
S3150800272042002000420075006C006B002000490042
S315080027306E00740065007200660061006300650043
S315080027404F70656E424C54002E2E2F2E2E2F2E2E95
S315080027502F536F757263652F41524D434D335F5347
S31508002760544D333246312F7573622E6300000000D4
S315080027700060000800200000030000000080000838
S31508002780002000000400000000A00008002000004F
S315080027900500000000C00008002000000600000038
S315080027A000E0000800200000070000000000010803
S315080027B0002000000800000000200108002000009A
S315080027C00900000000400108002000000A0000007F
S315080027D000600108002000000B00000000800108CE
S315080027E0002000000C00000000A0010800200000E6
S315080027F00D00000000C00108002000000E000000C7
S3150800280000E00108002000000F0000002E2E2F2EE9
S315080028102E2F2E2E2F536F757263652F41524D43FF
S315080028204D335F53544D333246312F4743432F764A
S311080028306563746F72732E63000000006D
S3150800283CD826000820000000E90300081104000847
S3150800284C810300088503000889030008D5030008DE
S3150800285CD9030008C5040008D5040008E5040008D7
S3150800286C0000000040000000AD10000855030008E9
S3150800287CAD100008AD100008AD100008AD1000082A
S3150800288CAD100008AD10000871030008EA26000810
S3150800289C090000009826000812000000AC26000863
S315080028AC04000000F82600081A000000B0260008EC
S315080028BC26000000980000201C00000014270008C1
S315080028CC2C000000030100001C03530045005200B5
S315080028DC310032003300340035003600370038003A
S315080028EC390030002D030008AD100008AD100008A3
S315080028FCAD100008AD100008AD100008AD100008AA
S3150800290C35030008AD100008AD100008AD1000081E
S3120800291CAD100008AD100008AD100008044D
S70508000000F2
